:020000040000FA
:04000000ABEF02F070
:0800080041EF0EF0116A156AC8
:10001000146E020E02D0146E030E066E1550115CA3
:1000200002E11450105C040ED8B0010ED8B4020ED8
:100030000614D8A4010E1200800E016EFE0ED5D853
:10004000010ED3D8750E116E300EE6D0016A018E06
:100050001F6EFE0ECAD81F50C8D0056A186E196AE6
:1000600000960550D8B40086050E046E270E156E56
:10007000100E0CD8030E156EE80E08D8156A640E23
:1000800005D8156A0A0E02D8185007D0146E1950F8
:10009000116E1850106E27D91050106E044E009635
:1000A000055003E0045CD8B007D01050D8A40096E7
:1000B00000B602D0300F99D012000096055003E12F
:1000C00000860A0E056E25C013F024C012F023C06E
:1000D00011F022C010F0046A1B6A1A6A196A0A0E2B
:1000E000186EA4D8042A0450055CD8A4F5D718507B
:1000F000D8A4009600A602D0052C03D01850300FCB
:1001000074D8052EE0D71200186E0450D8B412002F
:1001100018C0E9FF19C0EAFFEF50D8B4120065D843
:10012000184A192A0406F1D7046E055001E112009D
:1001300004505BD80506F9D7A66AA68E0900F550CB
:1001400002E002D8FBD712001D6E8A9600008A9446
:10015000939693940F0E93161D5000B21ED03A0E34
:10016000116E980E59D8330E1C6E29D8130E116ECD
:10017000880E52D824D8640E4ED821D8640E4BD89D
:10018000220E1C6E1CD8280E07D80C0E05D8060EA1
:1001900003D800821D5001D000801C6E00A00AD040
:1001A0008A9403080BE30AD8070E116ED00E34D8D8
:1001B000D88012000080FE0816E08A8400A000901B
:1001C0008A860F0E81161C50F00B8112000000D0A1
:1001D00000008A961C3A000000D0000000B0EFD763
:1001E000320E19D8D8801D50120001BEADD701A221
:1001F00005D001B003D001B2EE6E1200156A146E84
:10020000FF0E1426152200D0D8A01200030E116E86
:10021000E70E02D8F5D7116AFE0F106EE86A115A80
:10022000D8A012000000100600D0F8D713501B18F9
:10023000800BF46E13AE06D0D880000E1056115607
:10024000125613561BAE06D0D880000E18561956FB
:100250001A561B56146A156A166A176A286A296A9A
:100260002A6A2B6A1B501A101910181023E0200E4E
:10027000F36ED890103611361236133628362936DA
:100280002A362B361850285C195029581A502A58EB
:100290001B502B5809E31850285E1950295A1A5040
:1002A0002A5A1B502B5AD880143615361636173654
:1002B000F32EDFD7F4AE06D0D880000E14561556B4
:1002C0001656175614C010F015C011F016C012F0D3
:1002D00017C013F028C018F029C019F02AC01AF06E
:1002E0002BC01BF01200196A186A100EF36E11343D
:1002F000183619361450185C1550195805E3145067
:10030000185E1550195AD88010361136F32EEFD7D3
:100310001050120013C02BF012C02AF011C029F0A7
:1003200010C028F02A501802F3CF12F0F4CF13F0C7
:1003300029501902F3501226F450132228501A02A1
:10034000F3501226F45013222B501802F3501326A8
:100350002A501902F350132629501A02F35013267B
:1003600028501B02F350132628501802F3CF10F028
:10037000F4CF11F029501802F3501126F450122234
:10038000000E132228501902F3501126F4501222A5
:10039000000E13221200A66AA68E0900F55002E094
:1003A000EE6EFBD712002DC033F07F0E2C5C326E48
:1003B00002E2E86A4AD02D8E2C6A286A3250170869
:1003C000326E0CE2080E3226D8A03DD02DC02CF0A3
:1003D0002EC02DF02FC02EF02F6A0CD0080E325EEA
:1003E00008E32FC028F02EC02FF02DC02EF02D6A6C
:1003F000F5D73226325208E0D8902C322D322E32E8
:100400002F322832322EF8D72CB01DD031AC09D083
:1004100028AE07D02F2A05E12E2A03E12D2A01E17B
:100420002D2A2C502FC02CF02F6E2D502EC02DF0C9
:100430002E6E33AE06D0D880000E2C562D562E567A
:100440002F562C501200318AE8682C6E2D6E2E6EBD
:100450002F6E12002020202020202020000041505C
:10046000547265636F726465722076312E310000BC
:10047000496E73657274205344206F72204D4D4352
:1004800000004D422046696C657320200000504CEE
:100490004159202000005245434F5244000045522C
:1004A0004153452000004552524F5220696E207240
:1004B000652D696E697400005265636F7264696EC0
:1004C000672000004475726174696F6E20202030CF
:1004D000303A303000004552523A20436172642075
:1004E00046756C6C00004552523A204F7665727228
:1004F000756E00004E6F2066696C657320746F2006
:10050000706C61790000506C6179696E6720202001
:100510000000202030303A3030004552523A205509
:100520006E64657272756E00436F6E6669726D20DF
:100530004572617365004552523A20204E6F204645
:10054000696C65004552523A2046696C65206578B1
:10055000697374730000F86A400E316E006AAB6A0A
:100560000001070EB46E0F0EC16E40EF0EF0010ECB
:10057000695C09E3685002EE18F0E926000EEA22F1
:100580006AC0EFFF08D001EE18F06850E926000EAF
:10059000EA226AC0EFFF010E0101166F6828010E02
:1005A000D8B4691800010EE143D86152FDE10101A0
:1005B000166B686A696A552A000E5622572258221D
:1005C000000102D0684A692A1200686A696A6B529F
:1005D00012E1546A01EE18F05450E926000EEA22A6
:1005E000EF6A02EE18F05450E926000EEA22EF6A94
:1005F000542AF0E101D080D8120032EC08F05D06F8
:10060000000E5E5A53C010F05F5006EC00F0306EE2
:100610005E505D1002E0000E01D0010E3012EDE0E0
:100620005E505D1003E1010E606E01D0606A120041
:1006300001010E6B010E616E0001D890596A5534AC
:100640005A6E56345B6E57345C6E94928292580E9A
:10065000626E5CC063F05BC064F05AC065F059C064
:1006600066F067685F6A5D685E680DEC08F0C5DF7C
:10067000010E605C37E0FE0E676E2BEC08F0546AEA
:1006800001EE18F05450E926000EEA22EF50676E92
:100690002BEC08F0542AF4E1546A02EE18F054509E
:1006A000E926000EEA22EF50676E2BEC08F0542A80
:1006B000F4E167682BEC08F02BEC08F05F685D68EC
:1006C0005E6832EC08F053C0F2F097DF0F0EF217BD
:1006D000050EF25D07E1010E605C04E0616A949230
:1006E000828209D09492828201010E2B030E0E5D4C
:1006F0000001D8A0A1D7120001010E6B010E616E9E
:100700000001D890596A55345A6E56345B6E57348E
:100710005C6E94928292510E626E5CC063F05BC01C
:1007200064F05AC065F059C066F067680DEC08F0D7
:100730005F6A5D685E6861DF010E605C2DE0FE0E41
:100740005F6E5D685E6859DF010E605C25E0546A8B
:1007500032EC08F001EE18F05450E926000EEA22BF
:1007600053C0EFFF542AF4E1546A32EC08F002EE71
:1007700018F05450E926000EEA2253C0EFFF542A25
:10078000F4E132EC08F032EC08F09492828267686F
:100790002BEC08F0616A09D09492828201010E2B41
:1007A000030E0E5D0001D8A0ABD71200010E705CE5
:1007B00017E36F5002EE18F0E926000EEA22EF5020
:1007C000986F010E6F24226E000E7020236E22504F
:1007D00002EE18F0E926000EEA22EF50996F10D0D1
:1007E00001EE18F06F50E926000EEA22EF50986FE4
:1007F0006F2801EE18F0E926000EEA22EF50996FFB
:10080000120079508825226E7A508921236E000EBD
:100810008A21246E000E8B21256E2204F56F000EB6
:100820002358F66F000E2458F76F000E2558F86F06
:1008300088519A25726E89519B21736E8A519C2131
:10084000746E8B519D21756E7250F55D7350F65923
:100850007450F7597550F8597550F819D8B0800A86
:10086000D8A855D075C058F074C057F073C056F072
:1008700072C055F0010E6B6EA8DE6F6A706A020ED0
:10088000705CD8B03DD088519A250B6E89519B2160
:100890000C6E8A519C210D6E8B519D210E6E7250F3
:1008A0000B5C73500C5874500D5875500E587550A1
:1008B0000E18D8B0800A02E7000E01D0010E306E8B
:1008C000D890F935226EFA35236E22509E250B6E94
:1008D00023509F210C6E6FC010F070C011F00CC03F
:1008E00015F00B500BEC00F0301204E05FDF995173
:1008F000981110E0020E6F26C2E3702AD8A4BFD769
:10090000722A000E732274227522D8A09DD7010E80
:100910006C6E12008851725C9A6F895173589B6F8C
:100920008A5174589C6F8B5175589D6F6FC09EF0A3
:1009300070C09FF09AC0E7F0E66BD8909F31236EAD
:100940009E31226E2250E6272350E723F96BFA6B83
:100950009EC06FF09FC070F0020E705C0DE226DF4B
:100960009951981103E1F94BFA2B01D005D0020EF1
:100970006F26F2E3702AF0E1010EFB6FFC6B6C6AEC
:100980001200E56B716A080E715C1CE2010EE55DF8
:10099000010ED8A4000E306E00EEB2F07150EB5094
:1009A0000B6E010E0B52D8A4000E301209E0200E7F
:1009B000F36E00EEB2F07150F3CFEBFF010EE56F76
:1009C000712AE1E1E56B080E716E0B0E715C1FE29E
:1009D000010EE55D010ED8A4000E306E080E715CAC
:1009E00000EEBBF0EB500B6E010E0B52D8A4000EC4
:1009F00030120BE0080E715CBB0FE96E000EEA6A64
:100A0000EA22200EEF6E010EE56F712ADEE1120080
:100A1000B8DF826B836B84519025226E85519121C2
:100A2000236E000E9221246E000E9321256E220467
:100A3000F56F000E2358F66F000E2458F76F000E66
:100A40002558F86F93C075F092C074F091C073F0A0
:100A500090C072F07250F55D7350F6597450F759AA
:100A60007550F8597550F819D8B0800AD8A8ECD04C
:100A700075C058F074C057F073C056F072C055F08E
:100A8000010E6B6EE5EC02F06F6A706A020E705C2C
:100A9000D8B0D3D0716A200E715C26E271506F24F9
:100AA000F36F000E7020F46F010EF45D0EE3F3514E
:100AB00002EE18F0E926000EEA22EFCF0BF000EE6E
:100AC000BFF071500BC0EBFF0DD001EE18F0F351E9
:100AD000E926000EEA22EFCF0BF000EEBFF07150D6
:100AE0000BC0EBFF712AD7E101010153000112E1B4
:100AF000BF510B6E010E0B52D8A4000E306EBF51C9
:100B00000B6EE50E0B5C010ED8A4000E3012D8A4BB
:100B10009ED08CD0010E0101015D000133E1E56B37
:100B2000716A080E715C12E200EEBFF07150EB507A
:100B30000B6E00EEB2F07150EB500F6E0B500F5C6D
:100B400003E0010EE56F02D0712AEBE1080E716E31
:100B50000B0E715C13E200EEBFF07150EB500B6EA8
:100B6000080E715C00EEBBF0EB500F6E0B500F5C8B
:100B700003E0010EE56F02D0712AEAE1E553D8B433
:100B800066D054D0020E0101015D0001D8A44ED000
:100B9000CA510F6EF00E0F100B6E0C6A0B280C1062
:100BA000D8B444D0BF510B6E0B52D8B43FD0BF5114
:100BB0000B6EE50E0B5C3AE0CA510F6E1E0E0F1461
:100BC0000B6E0C6A0C500B1031E1824B832B010130
:100BD00007510001835D2AE1010106510001825D98
:100BE00025E1716A080E715C0CE200EEBFF07150F5
:100BF000EBCF0BF000EEB2F071500BC0EBFF712A9F
:100C0000F1E1080E716E0B0E715C0FE2080E715C63
:100C10000B6E00EEBFF07150EBCF0FF000EEBBF0AB
:100C20000B500FC0EBFF712AEEE111D0200E6F26A2
:100C3000D8A02CD7702AD8A429D7722A000E7322E4
:100C400074227522D8A006D7010E6D6E1200905145
:100C5000725CA66F91517358A76F92517458A86F28
:100C600093517558A96F6FC0AAF070C0ABF06D6A50
:100C70001200010EE45D09E3E35102EE18F0E926EB
:100C8000000EEA226EC0EFFF08D001EE18F0E3512B
:100C9000E926000EEA226EC0EFFF1200A4C0E3F0C6
:100CA000A5C0E4F0A0C0E7F0E66BD890A531236EB4
:100CB000A431226E2250E6272350E723E64BE72B90
:100CC000FE5303E1020EFD5D10E3E6C06EF0D1DFDE
:100CD000E34BE42BE7C06EF0CCDFE34BE42BE64BB9
:100CE000E72BFD07000EFE5BEBD712009AC0E7F082
:100CF000E66BD8909F31236E9E31226E2250E627FC
:100D00002350E723E6C06EF0B4DFE34BE42BE7C0EB
:100D10006EF0AFDF12006E68ACDFE34BE42BA9DFAF
:100D200012000101022B000E0323042305230251AC
:100D30000001ED5D010103510001EE590101045173
:100D40000001EF59010105510001F0590101055160
:100D50000001F019D8B0800A06E6ED2B000EEE2354
:100D6000EF23F0233D86B04BB12BB051805DB151E4
:100D70008159D8B020D1AC2B000EAD23AE23AF23C8
:100D8000EC2BEC51765CD8B011D13DB688D0E6C0E2
:100D900010F0E7C011F0126A136A1B6A1A6A010E9A
:100DA000196E186A16EC01F013C09DF012C09CF089
:100DB00011C09BF010C09AF0E6C09EF09F6BD890D7
:100DC0009E379F379A518825556E9B518921566EC3
:100DD0009C518A21576E9D518B21586E010E6B6E6E
:100DE000E5EC02F09EC06FF09FC070F0D6EC03F00F
:100DF00098C0E6F099C0E7F0FE0EE625226EFF0EE1
:100E0000E721236EFF0E246A2422256A252225C0AD
:100E100013F024C012F023C011F022C010F01B6A9E
:100E20001A6A196A76C018F08AEC01F013C0AFF0A4
:100E300012C0AEF011C0ADF010C0ACF09451AC27B0
:100E40009551AD239651AE239751AF23AFC058F0C3
:100E5000AEC057F0ADC056F0ACC055F0010E6B6E91
:100E6000E5EC02F0010EEC6FE6C010F0E7C011F007
:100E7000126A136A1B6A1A6A196E186A16EC01F074
:100E800013C09DF012C09CF011C09BF010C09AF0EE
:100E9000E6C09EF09F6BD8909E379F3786D0FB4B65
:100EA000FC2BFB51F95DFC51FA59D8B07AD09EC0A9
:100EB000A4F09FC0A5F09DC0A3F09CC0A2F09BC071
:100EC000A1F09AC0A0F0FBC0FFF0FCC000F1F9C097
:100ED000FDF0FAC0FEF001EC04F0010E6C5CD8B439
:100EE0001200A0518825DF6FA1518921E06FA25126
:100EF0008A21E16FA3518B21E26FE2C058F0E1C07B
:100F000057F0E0C056F0DFC055F0010E6B6EE5EC17
:100F100002F0C4DEEBDE18EC03F0A0518C25556E18
:100F2000A1518D21566EA2518E21576EA3518F2152
:100F3000586E18EC03F0FE0EE625226EFF0EE72138
:100F4000236EFF0E246A2422256A252225C013F071
:100F500024C012F023C011F022C010F01B6A1A6ADC
:100F6000196A76C018F08AEC01F013C0AFF012C015
:100F7000AEF011C0ADF010C0ACF09451AC2795515B
:100F8000AD239651AE239751AF23AFC058F0AEC0FA
:100F900057F0ADC056F0ACC055F06B6AE5EC02F00E
:100FA00002D0E64BE72B010EEC6F02D07CEC03F095
:100FB000010EB06FB16BF1C06AF0B7EC02F06C6A71
:100FC0001200010E0101016F000108EC05F0120092
:100FD000020E695C0BE3686A696A552A000E5622A4
:100FE00057225822010E6B6EE5EC02F0010E695C8F
:100FF00009E3685002EE18F0E926000EEA22EF50ED
:101000006A6E08D001EE18F06850E926000EEA2258
:10101000EF506A6E684A692A120062C0C9FFC7A011
:10102000FED7C9CF53F063C0C9FFC7A0FED7C9CF51
:1010300053F064C0C9FFC7A0FED7C9CF53F065C045
:10104000C9FFC7A0FED7C9CF53F066C0C9FFC7A06C
:10105000FED7C9CF53F067C0C9FFC7A0FED7C9CF1D
:1010600053F01200C968C7A0FED7C9CF53F01200D1
:10107000400EC76E9492949A949694889492828229
:10108000626863686468656866686768C6DFC5DF4C
:10109000640EFEEC00F094928292400E626E636ADF
:1010A000646A656A666A950E676EB7DF010E5F6EE9
:1010B0005D685E6AFDEC02F0010E605C05E19492F1
:1010C0008282010E616E12005468410E626E636A84
:1010D000646A656A666A6768A0DF5F6A5D685E6AFF
:1010E000FDEC02F05406010E6052D8A4000E306EE2
:1010F000010E5452D8A4000E3012E7E0545205E11C
:1011000094928282010E616E1200949282826768CC
:10111000A2DF686A696A616A1200010E0101165D48
:10112000000104E118EC03F06152FCE1A6519025A6
:10113000DF6FA7519121E06FA8519221E16FA95172
:101140009321E26FE2C058F0E1C057F0E0C056F0E2
:10115000DFC055F0010E6B6EE5EC02F01C0EAA2507
:10116000E36F000EAB21E46FEDC06EF039EC06F0DA
:10117000E34BE42BEEC06EF039EC06F0E34BE42BCE
:10118000EFC06EF039EC06F0E34BE42BF0C06EF0EC
:1011900039EC06F0160EAA25E36F000EAB21E46FC2
:1011A0005BD818EC03F03DA63CD09EC0A4F09FC0D5
:1011B000A5F09DC0A3F09CC0A2F09BC0A1F09AC076
:1011C000A0F0A0518825DF6FA1518921E06FA251C5
:1011D0008A21E16FA3518B21E26FE2C058F0E1C098
:1011E00057F0E0C056F0DFC055F0010E6B6EE5EC35
:1011F00002F0FBC0FDF0FCC0FEF04EEC06F08BEC04
:1012000006F018EC03F0A0518C25556EA1518D21EC
:10121000566EA2518E21576EA3518F21586E18EC35
:1012200003F0120012C122F0236A13C126F0276ACC
:10123000010E2616276A2750640DF3CF27F026509B
:10124000640DF3CF26F0F4502726225026246E6E2C
:1012500039EC06F0E34BE42B13C122F0236AD8905B
:101260002332223214C126F0276A050ED890263682
:101270002736E82EFBD7225026106E6E39EC06F08A
:10128000E34BE42B14C122F0236A233222322332AF
:101290002232233222321F0E231615C126F0276A6E
:1012A000030ED89026362736E82EFBD7225026107C
:1012B0006E6E39EC06F0E34BE42B10C123F0226A8A
:1012C000D8902332223223322232233222320101B9
:1012D0000F5122106E6E000139EC06F0E34BE42B47
:1012E00010C122F0236A23322232233222322332E7
:1012F00022321F0E231611C126F0276A140E26264D
:10130000000E2722D89026362736225026106E6EE1
:1013100039EC06F01200C6CFC6FFC68AA9DE61C04E
:1013200009F1010E0101095D000103E1010E6C6E7E
:101330001200586A576A566A556A010E6B6EE5ECE0
:1013400002F0010118510B6EEB0E0B5C010ED8A4DC
:10135000000E306E1A510B6E900E0B5C010ED8A46D
:10136000000E3016000103E0866B876B11D001017F
:1013700018510B6EE90E0B5C000103E1866B876B65
:1013800007D00201DE510F6E0FC086F00001876B9F
:1013900086C055F087C056F0576A586A010E6B6ECA
:1013A000E5EC02F0010123510001806F010124519D
:1013B0000001816F01012551766E2651776E27510C
:1013C000786E28517B6E29510001826F01012A51EC
:1013D0000001836F01012E51796E2F517A6E3851C1
:1013E0007C6E39517D6E3A517E6E3B517F6E7750E7
:1013F00000018625886F78508721896F000E8A6BDF
:101400008A238B6B77508625226E78508721236E36
:10141000000E246A2422256A795022248C6F7A5087
:1014200023208D6F000E24208E6F000E25208F6FDD
:10143000136A126A116A7BC010F079C018F07AC082
:1014400019F01A6A1B6A8AEC01F013C093F012C0FB
:1014500092F011C091F010C090F077508625226E66
:1014600078508721236E000E246A2422256A225098
:101470009027235091232450922325509323835166
:10148000200DF3CF85F08251200DF3CF84F0F4507E
:10149000852784C010F085C011F080C014F081C091
:1014A00015F073EC01F0846F11C085F08451902524
:1014B000946F85519121956F000E9221966F000EC9
:1014C0009321976F86517C24226E87517D20236E55
:1014D000000E7E20246E000E7F20256E2204556EA5
:1014E000000E2358566E000E2458576E000E2558D5
:1014F000586E9451555C226E95515658236E9651F4
:101500005758246E97515858256E2228556E000E54
:101510002320566E000E2420576E000E2520586E94
:1015200058C013F057C012F056C011F055C010F05B
:101530001B6A1A6A196A76C018F016EC01F013C01B
:1015400058F012C057F011C056F010C055F0010EFF
:101550005524EA6F000E5620EB6F00EEB2F0040E39
:10156000F76E540EF66ECBEC01F0EF6A00EEBBF0B6
:10157000200EEE6EEE6EEE6EEF6A010E01010F6F41
:10158000106F116B126B136B146B156B066B076B83
:101590006C6A000112000301186B00019D6B9C6BCB
:1015A0009B6B9A6B9E6B9F6BF96BFA6B01EC04F073
:1015B000010E6C5CD8B412000101016B000108EC53
:1015C00005F0010E6D5C03E1010E6C6E1200A65178
:1015D0009025DF6FA7519121E06FA8519221E16F13
:1015E000A9519321E26FE2C058F0E1C057F0E0C08A
:1015F00056F0DFC055F0010E6B6EE5EC02F0716A3B
:10160000200E715C0BE27150AA25E36F000EAB2136
:10161000E46F6E6A39EC06F0712AF2E1C1EC04F075
:10162000716A080E715C0FE27150AA25E36F000E1B
:10163000AB21E46F00EEB2F07150EB506E6E39ECFE
:1016400006F0712AEEE1080E716E0B0E715C10E26D
:101650007150AA25E36F000EAB21E46F080E715C98
:1016600000EEBBF0EB506E6E39EC06F0712AEDE146
:101670000B0EAA25E36F000EAB21E46F200E6E6EF9
:1016800039EC06F00D0EAA25E36F000EAB21E46FD6
:1016900012EC09F01A0EAA25E36F000EAB21E46FDD
:1016A000E6C06EF039EC06F0E34BE42BE7C06EF0D9
:1016B00039EC06F018EC03F0FE0EE625226EFF0E64
:1016C000E721236EFF0E246A2422256A252225C0E5
:1016D00013F024C012F023C011F022C010F01B6AD6
:1016E0001A6A196A76C018F08AEC01F013C0AFF0DC
:1016F00012C0AEF011C0ADF010C0ACF09451AC27E8
:101700009551AD239651AE239751AF23010EEC6F47
:10171000AFC058F0AEC057F0ADC056F0ACC055F0F9
:101720006B6AE5EC02F0B06BB16BF06BEF6BEE6BDC
:10173000ED6B0101056B046B036B026B3D86010EC3
:101740000301186F00011200E1EC07F06D5203E095
:10175000010E6C6E1200D951E66FDA51E76FDB5162
:10176000ED6FDC51EE6FDD51EF6FDE51F06FFE0E6D
:10177000E625226EFF0EE721236EFF0E246A242247
:10178000256A252225C013F024C012F023C011F0D1
:1017900022C010F01B6A1A6A196A76C018F08AEC27
:1017A00001F013C0AFF012C0AEF011C0ADF010C028
:1017B000ACF09451AC279551AD239651AE2397517F
:1017C000AF23010EEC6FAFC058F0AEC057F0ADC004
:1017D00056F0ACC055F06B6EE5EC02F0010E615CAA
:1017E00003E1010E6C6E1200B06BB16B0101056B71
:1017F000046B036B026BD8960001F0BFD88607E438
:10180000ED51EE11EF11F01102E03D9601D03D8651
:101810000101166B010E0001F96FFA6B6C6A120080
:101820003DB6ADD0B04BB12BB051805DB1518159B7
:10183000D8B086D0010E0101165D000106E118EC5A
:1018400003F06152FCE10101166B0001AC2B000EAC
:10185000AD23AE23AF23EC2BEC51765CD8B06DD02A
:10186000E6C010F0E7C011F0126A136A1B6A1A6A28
:10187000010E196E186A16EC01F013C09DF012C02B
:101880009CF011C09BF010C09AF0E6C09EF09F6BD8
:10189000D8909E379F379A518825556E9B51892144
:1018A000566E9C518A21576E9D518B21586E010EA8
:1018B0006B6EE5EC02F09EC06FF09FC070F0D6EC4E
:1018C00003F098C0E6F099C0E7F0FE0EE625226E20
:1018D000FF0EE721236EFF0E246A2422256A2522AB
:1018E00025C013F024C012F023C011F022C010F064
:1018F0001B6A1A6A196A76C018F08AEC01F013C0E4
:10190000AFF012C0AEF011C0ADF010C0ACF0945109
:10191000AC279551AD239651AE239751AF23AFC05D
:1019200058F0AEC057F0ADC056F0ACC055F0010E47
:101930006B6EE5EC02F0010EEC6F010EB06FB16B57
:10194000E8EC07F00101022B000E0323042305231A
:101950000001ED510101025D0001EE510101035949
:101960000001EF51010104590001F0510101055935
:1019700005510001F019D8B0800AD8B83D86120090
:10198000F96BFA6B79508825226E7A508921236E83
:10199000000E8A21246E000E8B21256E2204076E14
:1019A000000E2358086E000E2458096E000E2558AC
:1019B0000A6E8BC075F08AC074F089C073F088C05D
:1019C00072F07250075C7350085874500958755083
:1019D0000A5875500A18D8B0800A23E775C058F025
:1019E00074C057F073C056F072C055F0010E6B6EA4
:1019F000E5EC02F06F6A706A020E705C0CE2D6ECE5
:101A000003F09951981102E1F94BFA2B020E6F265F
:101A1000F3E3702AF1E1722A000E73227422752218
:101A2000D0E3F86B7AC0F7F079C0F6F0F56BEA51C5
:101A3000F55D226EEB51F659236E000EF759246EB8
:101A4000000EF859256E2204F56F000E2358F66F2C
:101A5000000E2458F76F000E2558F86FF551F95D08
:101A60000101026F0001F651FA590101036F000EE6
:101A70000001F7550101046F000E0001F855010146
:101A8000056F05C113F004C112F003C111F002C1CA
:101A900010F01B6A1A6A196A76C018F08AEC01F015
:101AA00013C005F112C004F111C003F110C002F11E
:101AB00005C113F004C112F003C111F002C110F00E
:101AC0001B6A1A6A196A020E186E16EC01F013C02E
:101AD00005F112C004F111C003F110C002F10001C0
:101AE0001200546A01EE18F05450E926000EEA2262
:101AF000EF6A02EE18F05450E926000EEA22EF6A6F
:101B0000542AF0E184519025226E85519121236E53
:101B1000000E9221246E000E9321256E2204076E82
:101B2000000E2358086E000E2458096E000E25582A
:101B30000A6E93C058F092C057F091C056F090C012
:101B400055F05550075C5650085857500958585092
:101B50000A5858500A18D8B0800A08E718EC03F061
:101B6000552A000E562257225822EBE38829556E3B
:101B7000000E8921566E000E8A21576E000E8B21B1
:101B8000586E79508825226E7A508921236E000E76
:101B90008A21246E000E8B21256E2204076E000E12
:101BA0002358086E000E2458096E000E25580A6E40
:101BB0005550075C565008585750095858500A5805
:101BC00058500A18D8B0800A08E718EC03F0552AD4
:101BD000000E562257225822EBE38C29556E000E38
:101BE0008D21566E000E8E21576E000E8F21586E7D
:101BF00079508C25226E7A508D21236E000E8E2115
:101C0000246E000E8F21256E2204076E000E2358CD
:101C1000086E000E2458096E000E25580A6E5550A5
:101C2000075C565008585750095858500A58585091
:101C30000A18D8B0800A08E718EC03F0552A000EFD
:101C4000562257225822EBE3F80E0101186F19694A
:101C50001A691B698BC058F08AC057F089C056F0CA
:101C600088C055F0000118EC03F08FC058F08EC00A
:101C700057F08DC056F08CC055F018EC03F01200F0
:101C80003BD0E9CF3AF0EACF3BF000019E923DA273
:101C900019D0C2B4FED7C4CFBEFFC28403EE19F080
:101CA0003450E9263550EA22BECFEFFF344A352AB8
:101CB00035943750355C05E13650345C02E1818261
:101CC0003D9215D03DA013D03550375C05E134501E
:101CD000365C02E181823D9003EE19F03650E92630
:101CE0003750EA22EFCFBEFF364A372A37943AC040
:101CF000E9FF3BC0EAFF11009268936A900E946E70
:101D00004F0EC16E800EC26E010E156EF40EFFEC0A
:101D100000F031C0F3FF0FEE80F0ED6AE950EA10F9
:101D2000FCE1EF6AF3CF31F0F29E829081908192D4
:101D30001CEC00F0040EF76E5E0EF66E9CEC00F0EC
:101D4000800E016EC00E26EC00F0040EF76E700ED1
:101D5000F66E9CEC00F081709390000EC66E000E43
:101D6000C76E000EC86E000EC96EC68A8BEC09F0F5
:101D70006CC03CF0C80EFEEC00F03C52ECE18190EF
:101D800081921CEC00F0456A3D84FADD05C141F00A
:101D900004C140F003C13FF002C13EF011EC12F06B
:101DA0003DA46FD0800E016E26EC00F0040E056E8F
:101DB00041C013F040C012F03FC011F03EC010F01F
:101DC0001B6A1A6A030E196EE80E186E16EC01F003
:101DD00013C025F012C024F011C023F010C022F06F
:101DE0005DEC00F0040EF76E820EF66E9CEC00F0D7
:101DF000020E056E43502EEC00F0800E016EC00EF8
:101E000026EC00F0430EA4EC00F06D0EA4EC00F004
:101E1000640EA4EC00F03A0EA4EC00F0200EA4EC4A
:101E200000F045520DE1040EF76E8E0EF66E9CEC3E
:101E300000F0800E016E0A0E056E200E94EC00F08C
:101E4000010E455C0DE1040EF76E960EF66E9CECED
:101E500000F0800E016E0A0E056E200E94EC00F06C
:101E6000020E455C0DE1040EF76E9E0EF66E9CECC4
:101E700000F0800E016E0A0E056E200E94EC00F04C
:101E80003D9480B819D0140EFEEC00F080A8FED767
:101E9000140EFEEC00F04528226E000E236A232269
:101EA00022C010F023C011F0030E146E156A73ECFB
:101EB00001F018C045F03D8480BA2BD08192140EF9
:101EC000FEEC00F080AAFED7140EFEEC00F04550A8
:101ED000106E02081DE3FA6AD8901036FA361036F2
:101EE000FA36040E10261F0EFA22FB6A000EFB22A1
:101EF0000500FF6A000EFF221F0EFE6E100EFD6E23
:101F00001050F96E80EF10F08BEF0FF0EBEF11F047
:101F10003D8446D7FFD7432A000EC66E000EC76E1B
:101F2000000EC86E000EC96EC68A8BEC09F06CC03C
:101F30003CF0010E3C5C0CE1800E016EC00E26EC04
:101F400000F0040EF76EA60EF66E9CEC00F0FFD7C4
:101F500000EEB2F0410EEE6E500EEE6E540EEE6ECE
:101F6000020E016E030E056E43502EEC00F0EF6A78
:101F700000EEBBF0410EEE6E530EEE6E520EEE6EA4
:101F8000EF6AE1EC07F06DC03CF03C5203E1B3EFC7
:101F900012F002D0CBEC0AF01CEC00F0800E016EC7
:101FA00026EC00F0040EF76EB80EF66E9CEC00F016
:101FB000090E046E196AB20E84EC00F0800E016EF8
:101FC000C00E26EC00F0040EF76EC40EF66E9CEC0C
:101FD00000F0260E486E496E486E4A6A4B6A4C6A9B
:101FE0004D6AE0D93D82C280C2848180E7D980AA4F
:101FF00070D03550375C03E13450365C27E074D93B
:1020000042C0F1F091EC06F06CC03CF0010E3C5C7B
:1020100010E18182DAD98DEC08F0800E016EC00EDD
:1020200026EC00F0040EF76ED60EF66E9CEC00F077
:10203000FFD74806000E495A4950481006E1260EBF
:10204000486E496E486E4A4A4B2A31D04D504B5C1F
:1020500003E14C504A5C2BE04AC04CF04BC04DF0C1
:102060004AC010F04BC011F03C0E146E156A73ECB0
:1020700001F04E6E4AC010F04BC011F03C0E146ED1
:10208000156A73EC01F018C04FF0800E016ECB0E94
:1020900026EC00F0020E056E4E502EEC00F03A0ECB
:1020A000A4EC00F0020E056E4F502EEC00F081A261
:1020B0000FD08BD98DEC08F0800E016EC00E26EC8F
:1020C00000F0040EF76EE60EF66E9CEC00F0FFD703
:1020D0008ED77BD98190140EFEEC00F080AAFED73B
:1020E000140EFEEC00F08DEC08F0C0EC0CF005C115
:1020F00041F004C140F003C13FF002C13EF01200C4
:10210000435211E1800E016EC00E26EC00F0040E69
:10211000F76EF40EF66E9CEC00F0070E156ED00E06
:10212000FFEC00F0120043C044F0A4D980AA14D000
:1021300080B811D0140EFEEC00F080A8FED7140E6B
:10214000FEEC00F04406445202E143C044F0140E99
:10215000FEEC00F08FD9EAD7140EFEEC00F080AA56
:10216000FED7140EFEEC00F0A4EC0BF06CC03CF0BB
:10217000010E3C5CD8B4EAD9C0D91CEC00F0800E4A
:10218000016E26EC00F0050EF76E060EF66E9CEC66
:1021900000F0090E046E196AB20E84EC00F0800E95
:1021A000016EC00E26EC00F04C0EA4EC00F0650EA3
:1021B000A4EC00F06E0EA4EC00F0200EA4EC00F0F5
:1021C000020E056E4E502EEC00F03A0EA4EC00F01C
:1021D000020E056E4F502EEC00F0050EF76E120E3B
:1021E000F66E9CEC00F0DED88180250E486E260E3F
:1021F000496E4A6A4B6A4C6A4D6A10EC0CF06AC030
:1022000042F0A1D83D80DAD83DB66BD034C038F06A
:1022100035C039F0384A392A39943750395C03E1EE
:102220003650385C12E010EC0CF06AC042F08BD8EB
:102230004806000E495A4950481006E1260E486EDD
:10224000496E486E4A4A4B2A31D04D504B5C03E1EF
:102250004C504A5C2BE04AC04CF04BC04DF04AC099
:1022600010F04BC011F03C0E146E156A73EC01F0C7
:102270004E6E4AC010F04BC011F03C0E146E156A41
:1022800073EC01F018C04FF0800E016ECB0E26ECFF
:1022900000F0020E056E4E502EEC00F03A0EA4EC4B
:1022A00000F0020E056E4F502EEC00F080BA09D0FF
:1022B000140EFEEC00F080AAFED7140EFEEC00F027
:1022C00010D081A20DD081D8800E016EC00E26ECF8
:1022D00000F0050EF76E1A0EF66E9CEC00F0FFD7BC
:1022E00093D773D88190120037A214D037A009D0A9
:1022F00006EE19F03650E926000EEA22EF50426E43
:1023000008D005EE19F03650E926000EEA22EF500B
:10231000426E13D037A009D004EE19F03650E926EA
:10232000000EEA22EF50426E08D003EE19F036504C
:10233000E926000EEA22EF50426EF29E364A372A14
:102340003794F28E120035A214D035A009D006EED3
:1023500019F03450E926000EEA2242C0EFFF08D0FF
:1023600005EE19F03450E926000EEA2242C0EFFFD4
:1023700013D035A009D004EE19F03450E926000E30
:10238000EA2242C0EFFF08D003EE19F03450E926EC
:10239000000EEA2242C0EFFFF29E344A352A3594FD
:1023A000F28E1200346A356A366A376A0C0EBD6ED8
:1023B000CB68800EBE6E180ECA6E12009E92CC6A5A
:1023C0009D82F28CF28ECA841200CA949D929E92D3
:1023D0003D923D901200800E016EC00E26EC00F082
:1023E000050EF76E280EF66E9CEC00F080BAFED754
:1023F000140EFEEC00F080AAFED7140EFEEC00F0E6
:102400009390818071EC0DF0C0EC0CF005C141F0AF
:1024100004C140F003C13FF002C13EF093908190AF
:102420001200010E436E640E435C23E200EEB2F034
:10243000410EEE6E500EEE6E540EEE6E020E016EFA
:10244000030E056E43502EEC00F0EF6A00EEBBF079
:10245000410EEE6E530EEE6E520EEE6EEF6AE1EC32
:1024600007F06DC03CF03C5202E043061200432AE4
:10247000DAE1120000EEB2F0410EEE6E500EEE6E9A
:10248000540EEE6E020E016E030E056E44502EECDD
:1024900000F0EF6A00EEBBF0410EEE6E530EEE6EF2
:1024A000520EEE6EEF6AA4EC0BF06CC03CF0010E25
:1024B0003C5CD8B44BD821D8800E016EC00E26ECFF
:1024C00000F0090E046E196AB20E84EC00F0200EC2
:1024D000A4EC00F0A4EC00F0020E056E4E502EECC1
:1024E00000F06D0EA4EC00F0020E056E4F502EECC5
:1024F00000F0730EA4EC00F01200F0C013F0EFC077
:1025000012F0EEC011F0EDC010F01B6A1A6A260E30
:10251000196E186E16EC01F010C046F011C047F0AD
:1025200046C010F047C011F03C0E146E156A73ECF3
:1025300001F04E6E46C010F047C011F03C0E146E14
:10254000156A73EC01F018C04FF01200800E016E96
:10255000C00E26EC00F0050EF76E360EF66E9CEC03
:1025600000F08182FFD7800E016EC00E26EC00F0D5
:10257000050EF76E440EF66E9CEC00F08182FFD7DC
:042580000300FED77F
:020000040030CA
:03000100061E0ECA
:020005008381F5
:060008000FC00FE00F40E5
:00000001FF
